:0CFCC100011200010C00010B00010E00FC
:10FC290012F8FA12FD3812FDB2E50CB4FF14E51909
:10FC3900D39400400DD5190AE47833F67F0AFE12F1
:10FC4900FD957837E6600712FC66E47837F620B050
:0DFC5900087837E6700312FA1B050C80C90D
:10F8FA00C2087580FF43BF027B007A0079087F0047
:10F90A007EEE12FD89AD08E4FFFE12FD7C7B007AD3
:10F91A000079097F017EEE12FD89AD097F017E0023
:10F92A0012FD7C7B007A0079137F027EEE12FD893C
:10F93A00AD137F027E0012FD7C7B007A0079147F72
:10F94A00037EEE12FD89AD147F037E0012FD7C7BDF
:10F95A00007A0079117F047EEE12FD89AD117F04D1
:10F96A007E0012FD7C7B007A00790F7F057EEE1205
:10F97A00FD89AD0F7F057E0012FD7C7B007A007940
:10F98A001B7F067EEE12FD89AD1B7F067E0012FDEF
:10F99A007C7B007A0079157F077EEE12FD89AD1512
:10F9AA007F077E0012FD7C7B007A00790A7F087E41
:10F9BA00EE12FD89AD0A7F087E0012FD7C7B007A7B
:10F9CA0000790D7F097EEE12FD89AD0D7F097E005B
:10F9DA0012FD7C7D1F7F0B7E0012FD7C7B007A006E
:10F9EA0079107F107EEE12FD89AD107F107E001215
:10F9FA00FD7CE5D85408F522E510B47F0302FDB278
:10FA0A00E522B4080402020022E522600302020091
:01FA1A0022C9
:04FDB200759FA72270
:0BFD9500EF1FAC0670011E4C70F62240
:10F28C0000C1814001C0804101C0804100C181406A
:10F29C0001C0804100C1814000C1814001C080415A
:10F2AC0001C0804100C1814000C1814001C080414A
:10F2BC0000C1814001C0804101C0804100C181403A
:10F2CC0001C0804100C1814000C1814001C080412A
:10F2DC0000C1814001C0804101C0804100C181401A
:10F2EC0000C1814001C0804101C0804100C181400A
:10F2FC0001C0804100C1814000C1814001C08041FA
:10F30C0001C0804100C1814000C1814001C08041E9
:10F31C0000C1814001C0804101C0804100C18140D9
:10F32C0000C1814001C0804101C0804100C18140C9
:10F33C0001C0804100C1814000C1814001C08041B9
:10F34C0000C1814001C0804101C0804100C18140A9
:10F35C0001C0804100C1814000C1814001C0804199
:10F36C0001C0804100C1814000C1814001C0804189
:10F37C0000C1814001C0804101C0804100C1814079
:10F38C0000C0C101C30302C2C60607C705C5C40439
:10F39C00CC0C0DCD0FCFCE0E0ACACB0BC90908C8A9
:10F3AC00D81819D91BDBDA1A1EDEDF1FDD1D1CDC99
:10F3BC0014D4D515D71716D6D21213D311D1D01009
:10F3CC00F03031F133F3F23236F6F737F53534F4F9
:10F3DC003CFCFD3DFF3F3EFEFA3A3BFB39F9F83869
:10F3EC0028E8E929EB2B2AEAEE2E2FEF2DEDEC2C59
:10F3FC00E42425E527E7E62622E2E323E12120E0C9
:10F40C00A06061A163A3A26266A6A767A56564A4B8
:10F41C006CACAD6DAF6F6EAEAA6A6BAB69A9A86828
:10F42C0078B8B979BB7B7ABABE7E7FBF7DBDBC7C18
:10F43C00B47475B577B7B67672B2B373B17170B088
:10F44C005090915193535292965657975595945478
:10F45C009C5C5D9D5F9F9E5E5A9A9B5B99595898E8
:10F46C00884849894B8B8A4A4E8E8F4F8D4D4C8CD8
:10F47C004484854587474686824243834181804048
:10FCCD000116FF011D0101330001179601380001D6
:05FCDD003400011B00D2
:10FD3800C292E47833F67837F6E51B6003B4FF0324
:04FD4800751BFE2207
:0DFD6F00C292E47833F67837F675179622C5
:09FDA000D2927F0A7E0002FD955B
:10FA1B00E4F520D2087F04FE12FD95C208A2B09235
:10FA2B0000D2087F037E0012FD95C208A2B092019E
:10FA3B00D2087F037E0012FD95C208A2B09202D2BB
:10FA4B00087F037E0012FD95C208A2B09203D20874
:10FA5B007F037E0012FD95C208A2B09204D2087FEC
:10FA6B00037E0012FD95C208A2B09205D2087F0357
:10FA7B007E0012FD95C208A2B09206D2087F037ECB
:10FA8B000012FD95C208A2B09207D2087833E6C3E4
:10FA9B0094965007E6062439F8A620C2087833E678
:10FAAB00FFB517057837760122EF64077020783A97
:10FABB00E6FE64036004EEB4060475170822EEB488
:10FACB001008783FE62409F5172275179622EFB434
:10FADB00010475191922EFB40309783AE6B4190336
:04FAEB007517062263
:10FC97007832E6FF7E15D208C2B1DEFEE4FDEF132F
:10FCA70092B1EFC313FF7E12DEFE0DBD08F0D2B195
:0AFCB7007F087E0012FD95C20822AE
:10FC660012F7C9500C12FDA012FDA912F48C12F65F
:10FC76005612FD6FE516B40117E4FD7F107EEE12F5
:10FC8600FCE7AD1B7F067EEF12FCE7759F8080FECA
:01FC9600224B
:10F7C9007833E665176002C3227839E6FFF4600AE8
:10F7D900EF651B6005EF6002C322783AE664197091
:10F7E9007AFB7A0079397D0412FBA58E228F237862
:10F7F9003DE6FE08E67C002400FFEC3EFEEF6523B3
:10F809007003EE65226002C322783CE6FF18E6FE2B
:10F81900C39F4004AD078002AD06EEC39F4004AF0D
:10F82900068000E51BC39D4006E51BD39F4002C32C
:10F8390022AF0C7E0012FC1F12FBE87C007D1E1219
:10F84900FB1A8D25E4F524E524C39525500B7F6427
:10F859007E0012FD95052480EED322783AE6FF64F6
:10F8690003600CEF64066007EF64106002C322783E
:10F879003BE6FE08E67C002400FFEC3EFEEF640A4E
:10F889004E703B783AE6B4030C12FBE87C007D0528
:10F8990012FB1A8D1CE51C64016002C32212FBE8ED
:10F8A9007C007D1412FB1A8D25E4F524E524C3950B
:10F8B90025500B7F647E0012FD95052480EE7B00A8
:10F8C9007A007939E51724FEFD12FBA58E228F23D4
:10F8D90074372517F8E6FE74382517F8E67C0024F6
:06F8E90000FFEC3EFEEF03
:0BF8EF00B52306EEB52202D322C3228F
:10F65600E4F525783AE6B4061AE4F5257439252545
:10F66600F8E6FF12FC9B12FDB20525E525C39408BA
:10F6760040EA22783AE66403600302F75C08E6FE95
:10F6860008E67C002400F523EC3EF522783EE6F5FC
:10F69600247839E6FF12FC9B7839E6FF12FD2278C2
:10F6A6003AE6FF12FC9B783AE6FF12FD22E5242596
:10F6B600E0FF12FC9BE52425E0FF12FD22E525C3B1
:10F6C6009524400302F74FE4FF12FC9BE4FF12FD72
:10F6D60022E51DB47B167E00E5232525FFEE3522A7
:10F6E600FE7B007A00792612FD89804E7E00E52396
:10F6F6002525FFEE3522FEC3EF940CEE9400500B49
:10F706007B007A00792612FD4C802F7E00E52325AA
:10F7160025FFEE3522FEEF64204E700585BF26805C
:10F7260019EF642D4E7005851D26800EEF64304E50
:10F7360070058518268003752601AF2612FC9BAF3F
:10F746002612FD22052502F6C312FC977835E6FF40
:10F7560012FC9B02FDB2783AE66410702CF5257413
:10F76600392525F8E6FF12FC9B74392525F8E6FFB6
:10F7760012FD220525E525C3940640E312FC977881
:10F7860035E6FF12FC9B02FDB2783AE66419703248
:03F7960018E6FF73
:10F7990012FC9B7839E6FF12FD22783AE6FF12FC4B
:10F7A9009B783AE6FF12FD22AF1B12FC9BAF1B129E
:10F7B900FD2212FC977835E6FF12FC9B12FDB2225E
:10F48C00783AE664067064783CE6FFB406117E00B8
:10F49C00783EE6FD12FD7C783EE6F51B02F5EA7837
:10F4AC003CE6B40A1CE51C6401600302F5EA783EF4
:10F4BC00E6FD7F067E0012FD7C783EE6F51B02F52C
:10F4CC00EA783CE6FFB410117E00783EE6FD12FDB2
:10F4DC007C783EE6F51602F5EA783CE6642D60038E
:10F4EC0002F5EA783EE6F51D02F5EA783AE6641094
:10F4FC00600302F5EA783EE6F52A08E6FD783BE67D
:10F50C00FCFE08E6F97A002400F525EA3EF5248C89
:10F51C00288929E52A6D7033F526F527C3E527954B
:10F52C002AE5269400505A74402527F8E6F523E581
:10F53C00252527FFE5243526FEAD2312FCE712FD19
:10F54C00B20527E52770D5052680D1E4F526F527E9
:10F55C00C3E527952AE52694005026E52725E024C7
:10F56C0041F8E6F523E5252527FFE5243526FEADF4
:10F57C002312FCE712FDB20527E52770D305268080
:10F58C00CF783806E6640870557834E675F002A436
:10F59C002411FFE5F034EEFEE4FD12FCE77834E6CE
:10F5AC0075F002A42412FFE5F034EEFEE4FD12FC2B
:10F5BC00E7783406E675F002A42411FFE5F034EE8A
:10F5CC00FEAD2812FCE77834E675F002A42412FF95
:10F5DC00E5F034EEFEAD2912FCE7E47838F6E516DA
:10F5EC00B47F0BE47838F67834F675167E22E5167F
:10F5FC00B43F18E4F522AF2212FD0A12FDB2052227
:10F60C00E522C3946440EF75163E22E516B4330A26
:10F61C0012FDB212FD5F75163422E516B41F2212CC
:10F62C00FDB27D1F7F107EEE12FCE77DF07F117E18
:10F63C00EE12FCE77DF07F127EEE12FCE775161ED3
:0AF64C0022E516B4010312FDB222FC
:09FDA900783576FF783276FF22EE
:10FD22007832E66FFF90F28C937835667932F7EF8E
:06FD320090F38C93F62211
:10FBA5008B268A2789288D29752A00752BFF7DFFCD
:10FBB500AF291529EF6026AB260528E528AA277069
:10FBC50002052714F912FAEF652BFF90F28C936D5D
:10FBD500752A00F52BEF90F38C93FD80D3E52BFE72
:03FBE500EDFF220F
:04FCE20041000000DD
:10FCE7008E2B8F2C8D2D12FDB275F65575F6AA75D4
:10FCF700F65575BF04852DF6E52BF5F4852CF575BE
:03FD0700F7802260
:10FD0A0075F65575F6AA75F65575BF04EF25E0F533
:08FD1A00F4E4F5F575F782220F
:10FD5F0075F65575F6AA75F65575BF0475F78322B6
:0BFD89008F828E83E49312FB087F0141
:01FD9400224C
:0DFD7C0074002FF582E43400F583EDF022D1
:10FD4C0074002FF582E43400F583E012FB0812FAFC
:03FD5C00EFFF2294
:01F000001FF0
:0300000002F20009
:0CF20000787FE4F6D8FD7581CE02F2475D
:10FAEF00BB010689828A83E0225002E722BBFE0215
:09FAFF00E32289828A83E4932248
:10FB0800BB010689828A83F0225002F722BBFE01DC
:02FB1800F322D6
:10FB1A00C2D5EC30E709B2D5E4C39DFDE49CFCEE06
:10FB2A0030E715B2D5E4C39FFFE49EFE12FB50C333
:10FB3A00E49DFDE49CFC800312FB5030D507C3E42E
:06FB4A009FFFE49EFE2275
:10FBE800AC2EAD2FAE30AF31780FEFA2E2EC20E6AD
:10FBF80001B35D5E5FF47004FCFDFEFFEF13FFEEE2
:10FC080013FEED13FDEC13FCD8E08C2E8D2F8E30F7
:10FC18008F31EE547FFE228E2E8F2FE4F530F53192
:01FC280022B9
:10F20C0002FC29E493A3F8E493A34003F68001F2F3
:10F21C0008DFF48029E493A3F85407240CC8C33303
:10F22C00C4540F4420C8834004F456800146F6DFD2
:10F23C00E4800B010204081020408090FCC1E47EA5
:10F24C00019360BCA3FF543F30E509541FFEE493C7
:10F25C00A360010ECF54C025E060A840B8E493A38E
:10F26C00FAE493A3F8E493A3C8C582C8CAC583CAB9
:10F27C00F0A3C8C582C8CAC583CADFE9DEE780BE71
:01FCE600001D
:10FB5000BC000BBE0029EF8DF084FFADF022E4CC99
:10FB6000F875F008EF2FFFEE33FEEC33FCEE9DEC62
:10FB7000984005FCEE9DFE0FD5F0E9E4CEFD22EDA8
:10FB8000F8F5F0EE8420D21CFEADF075F008EF2FF2
:10FB9000FFED33FD4007985006D5F0F222C398FDE3
:05FBA0000FD5F0EA2280
:00000001FF
